:1000000097C0AFC0AEC0ADC0B3C0ABC0AAC0A9C09E
:10001000A8C0A7C0A6C0A5C0A4C0A3C0A2C0A1C0BC
:10002000A0C09FC09EC0C7C0BCC0C1C0C7C0BFC029
:10003000C5C0BDC0C3C0BBC0C1C0B9C0BFC0B7C0D0
:10004000BDC0B5C0BBC0B3C0B9C0C7C0CAC00A0D2F
:100050000A0D24505352463130302C312C34383074
:10006000302C382C312C302A30450A0D2450535274
:10007000463130332C30352C30302C30312C30316F
:100080002A32300A0D24505352463130332C30344A
:100090002C30302C30302C30302A32310A0D2450A4
:1000A0005352463130332C30332C30302C30302CFE
:1000B00030302A32360A0D24505352463130332C18
:1000C00030322C30302C30302C30302A32370A0D80
:1000D00000000A0D0A0D24504D544B3331342C309E
:1000E0002C302C312C312C302C302C302C302C302E
:1000F0002C302C302C302C302C302C302C302C3020
:100100002C302C302A32380A0D24504D544B3232C8
:10011000302C313030302A31460A0D24504D544BAA
:100120003235312C343830302A31340A0D00000099
:1001300011241FBECFEDCDBF10E0A0E6B0E0EEE78A
:10014000F3E002C005900D92A636B107D9F710E092
:10015000A6E6B0E001C01D92AA36B107E1F77AD059
:100160000CC14ECF89B7806489BF82E08EBD0895EF
:100170001F920F920FB60F9211248F939F93EF93BC
:10018000FF938AB59BB58C599F4F9BBD8ABD8091CB
:100190006900E82FF0E0E431F10580F5ED5EFF4FF6
:1001A0000994C098C19A809169008F5F25C08091A1
:1001B000680087FDF6CFC09AC198F5CF809168009E
:1001C00087FF03C0C09AC19802C0C098C19A8091AD
:1001D0006800880F80936800E6CFC098C19A83E1D9
:1001E0000BC0C09AC1985F9B06C08CB18093680019
:1001F0001092690003C082E18093690080916600DB
:1002000090916700892B49F080916600909167007A
:1002100001979093670080936600FF91EF919F9103
:100220008F910F900FBE0F901F9018958CB901C041
:1002300000005E9BFDCF5E9A0895909367008093C7
:10024000660001C000008091660090916700892BD4
:10025000C9F70895DF93CF9300D000D00F92CDB7A8
:10026000DEB7B89AB99A899AC79AC69A12B887E639
:1002700089B986E083B988E18AB989B7806489BF82
:1002800082E08EBD7894DE011196E0E6F0E085E034
:1002900001900D928150E1F780E197E29093670021
:1002A0008093660001C00000809166009091670015
:1002B000892BC9F7B79927C0DE01119648EE53E0A4
:1002C0009E012A5F3F4F12B88C9189B95093670005
:1002D0004093660001C00000809166009091670025
:1002E000892BC9F7EEE4F0E007C08CB901C000002B
:1002F0005E9BFDCF31965E9A84918823B1F711966B
:10030000A217B30701F7B69927C0DE01119648EE90
:1003100053E09E012A5F3F4F12B88C9189B95093E8
:1003200067004093660001C00000809166009091D4
:100330006700892BC9F7E2EDF0E007C08CB901C076
:1003400000005E9BFDCF31965E9A84918823B1F7C1
:100350001196A217B30701F787E689B988EE93E0F3
:10036000909367008093660001C000008091660052
:0E03700090916700892BC9F7FFCFF894FFCF5B
:06037E006733190C0800B2
:00000001FF
